:100000000C9496010C94BE010C94BE010C94BE019C
:100010000C94BE010C94BE010C94BE010C94BE0164
:100020000C94BE010C9437030C94EC230C949E2288
:100030000C94BE010C94BE010C94BE010C94BE0144
:100040000C94540A0C94BE010C94BE010C94BE0195
:100050000C94BE010C94BE010C94BE010C94BA1A0F
:100060000C94BE010C94931F0C94D61F0C94BE01EB
:100070000C94BE010C94BE010C94BE010C94BE0104
:100080000C94BE010C94BE010C94BE010C94BE01F4
:100090000C94BE010C94BE010C94BE010C94BE01E4
:1000A0000C94BE010C94BE010C94BE012D133313AD
:1000B000391340134E1370138E13C31BC61BB91B89
:1000C000BD1BE71BE71BE71BCA1BCE1BD21BD81BA4
:1000D000DC1BE71BE21B434C49206E6F74206176EA
:1000E00061696C61626C652C2075736520636F6E4D
:1000F000666967757261746F72210000000002000A
:10010000080E0000030401000B00000000000000C6
:100110000000000000000000000408020110408000
:1001200040102040804080080204018040201002DE
:10013000011080102040400404040404030405025C
:100140000202020403020202020606060606060472
:100150000402020204000000002300260029002CF3
:10016000002F0000000000250028002B002E003189
:100170000000000000240027002A002D00300008A5
:100180000B0002020201000904000001020200004B
:1001900005240010010524010101042402060524A0
:1001A0000600010705810310004009040100020A4E
:1001B000000000070502024000000705830240001E
:1001C0000000C18081C112010002020000404123F1
:1001D000368000010102000112010002000000400F
:1001E0004123368000010102000118034100720022
:1001F0006400750069006E006F0020004C004C0028
:1002000043002203410072006400750069006E0023
:100210006F0020004C0065006F006E0061007200EE
:1002200064006F00040309040000000000000000E7
:100230002A2B280000000000000000000000000041
:1002400000000000000000002C9EB4A0A1A2A43475
:10025000A6A7A5AE362D3738271E1F20212223241E
:100260002526B333B62EB7B89F8485868788898ABA
:100270008B8C8D8E8F909192939495969798999A56
:100280009B9C9D2F3130A3AD350405060708090A54
:100290000B0C0D0E0F101112131415161718191A36
:1002A0001B1C1DAFB1B0B500090402000103000022
:1002B00000092101010001226500070584034000B7
:1002C0000105010902A1010901A100850105091922
:1002D000012903150025019503750181029501751A
:1002E00005810305010930093109381581257F751C
:1002F0000895038106C0C005010906A10185020514
:100300000719E029E7150025017501950881029577
:1003100001750881039506750815002565050719FF
:100320000029658100C0741DC420882511241FBECA
:10033000CFEFDAE0DEBFCDBF12E0A0E0B1E0ECEB42
:10034000FDE402C005900D92AA35B107D9F715E07A
:10035000AAE5B2E001C01D92AC31B107E1F713E0AC
:10036000CCE2D3E004C02297FE010E945126C6329F
:10037000D107C9F70E9400210C94DC260C940000E0
:1003800080910008909101088737974709F0A89558
:100390000895DC01ED91FC910190F081E02D09952B
:1003A00008952091A0033091A103382748E0C901A6
:1003B000880F991F37FF06C09C0151E2252750E1A5
:1003C000352701C09C01415091F73093A103209340
:1003D000A003089588E38093A20380E092ECA1E05B
:1003E000B0E08093A3039093A403A093A503B093DC
:1003F000A60387E08093AF0380EC9AECA9E8B6E30C
:100400008093A7039093A803A093A903B093AA0392
:1004100085E08093B0038DEE9EEFADEABEED809354
:10042000AB039093AC03A093AD03B093AE03E1EBA9
:10043000F3E080E090E0863028F4DC01AC5DBD4F55
:100440002C9101C020E0219301968831910599F704
:1004500082E08093C9038AE08093CA03089580EC08
:1004600097EFAAEBB7E38093E7039093E803A09399
:10047000E903B093EA0380E090E0A0E0B0E5809368
:10048000EB039093EC03A093ED03B093EE03EFEE38
:10049000F3E080E081938F5F8031E1F70895A0E081
:1004A000B0E0E5E5F2E00C941A26D82F0E94101B6C
:1004B0006115710581059105C9F30E94BD26109251
:1004C000AB031092AC031092AD031092AE03C4E0E4
:1004D000812C912C54018A94C090AB03D090AC0332
:1004E000E090AD03F090AE03FE2CED2CDC2CCC2480
:1004F0000E94B826A50194010E94F9256C0D7D1D6E
:100500008E1D9F1D6093AB037093AC038093AD036E
:100510009093AE03C15001F7DD2309F450C001EB05
:1005200013E0E801A12CB12C62E3C62ED12CE12C02
:10053000F12C8881882309F442C0B39419F40E94F5
:10054000EA013DC00E94B826A70196010E94F92544
:10055000E1E0E60FA1EBB3E08A2F801B8A1520F4BF
:100560008D918E13F9CFE9CF2091B00330E0A0E157
:10057000B7E20E9491259B01AC01AE2FB0E00E9432
:10058000A0254090A7035090A8036090A903709005
:10059000AA03640D751D861D971D4090E7035090BA
:1005A000E8036090E9037090EA0346165706680670
:1005B000790618F2E993A39488E1A812BACFCDB7CF
:1005C000DEB7E0E10C94362680919F03813019F468
:1005D00082E080939F0380919F03833019F484E02D
:1005E00080939F03089588E08093C10061E08AE0D2
:1005F0000E94E81B60E08AE00E94211C0895009799
:10060000C9F09C0140E050E068E478EE81E090E0C1
:100610000E94F9252F3F31054105510529F020F0B1
:100620002FEF30E040E050E02093D1008091C000F7
:10063000806103C08091C0008F7E8093C0000895C8
:10064000219A229A239860E08BE00E94E81B61E0E7
:100650008CE00E94E81B0895EBE6F0E08081806862
:100660008083E8E6F0E080818160808308951F92B6
:100670000F920FB60F9211242F933F934F935F93D6
:100680006F937F938F939F93AF93BF93EF93FF935A
:100690001F9B0E94E402FF91EF91BF91AF919F9148
:1006A0008F917F916F915F914F913F912F910F901B
:1006B0000FBE0F901F901895A1E0B0E0E2E6F3E0C6
:1006C0000C9427261FB791E090939E03F89489839A
:1006D0000E94C00198E1909360008981809360003E
:1006E00081110E94C0011FBF2196E3E00C944326B4
:1006F0008F929F92AF92BF92CF92DF92EF92FF9232
:10070000CF93FC01C0A5EC2FE770F0E0E45EFD4F55
:10071000A081B0E0C7FF03C024E130E002C02FE0B9
:1007200030E0FC0197A183E1989FF0011124E25C85
:10073000FE4F80809180A280B380A20FB31F20E47F
:100740003FE14DE750E00E94AB25A50194010E94D6
:10075000D7258C2F887149F469017A01E0EDCE0E1E
:10076000E7E0DE1EE11CF11C1BC0C7FF05C060E412
:100770007AE88CE29EE004C060E07EEE8AEB9BE0CB
:1007800069017A01F8EBCF0EFBE0DF1EE11CF11CE2
:10079000A50194010E94D725C20ED31EE41EF51EAA
:1007A000C701B60169517C4F8F4F9F4F28EE33E050
:1007B00040E050E00E94D725A8EEB3E00E94A025BB
:1007C000CF91FF90EF90DF90CF90BF90AF909F9030
:1007D0008F9008958F3F910551F048F0811522E0E8
:1007E000920738F08115934030F482E0089580E05C
:1007F000089581E0089583E00895A0E0B0E0E3E08B
:10080000F4E00C942326EB018A01B82FB695A0E002
:1008100028813981F80120832A813B8121832C8121
:100820003D8122832E813F812383688179814A81A2
:100830005B812C813D81EE81FF819F2F9295990FE5
:10084000990F907C272F2370922B252F2370220F36
:10085000220F922B232F23702295207F922BF801B9
:1008600094830B5F1F4F2896AF5FBA1788F680FFFF
:1008700024C0888199810E94EA03D82E8A819B81B5
:100880000E94EA03E82E8C819D810E94EA03F82EE3
:100890008E819F810E94EA03F0E4DF9EA001112473
:1008A00090E1E99E90011124242B282BE4E0FE9E88
:1008B000B0011124262BF8012083CDB7DEB7E7E085
:1008C0000C943F26803223E0920708F1883E23E013
:1008D000920740F48F519340E4E096958795EA950E
:1008E000E1F70895803D27E0920718F48C5D93406E
:1008F0000895883928E0920768F4885C974074E08E
:10090000969587957A95E1F78D509C4F089580E0F4
:1009100090E008958FEF93E008958C30910540F4B6
:10092000A4E0880F991FAA95E1F7885D9C4F089570
:10093000843F23E0920718F484529C4F0895811558
:1009400024E0920740F48657934FF4E0880F991FF4
:10095000FA95E1F7089580E998E008959C013695AD
:10096000279525753575821B930B9C012373337373
:10097000969587959695879583739373820F931FAA
:100980009C0154E0369527955A95E1F7280F391FB9
:100990002F703F7041E051E0249FC001259F900DD2
:1009A000349F900D1124892F08952998882319F0D8
:1009B00000002A9A02C000002A980000299A00002C
:1009C0000895299A000083B12998000083FB8827A5
:1009D00080F90895CF93DF93D82F5E9A29985E9877
:1009E000C8E08D2F80780E94D504DD0FC150C9F773
:1009F0002998DF91CF9108958F770E94EA04089596
:100A0000CF93DF93D82FC8E08D2F80780E94D50434
:100A1000DD0FC150C9F72998DF91CF910895CF9389
:100A2000DF932998C8E080E0D82FDD0F0E94E10411
:100A30008D0FC150C9F7DF91CF9108950E94FC043A
:100A40000E940F055E9A0895A1E0B0E0EAE2F5E0A9
:100A50000C942826806869830E94EA046981862FA5
:100A60000E9400055E9A2196E2E00C944426CF9302
:100A7000C091AB03C827E82FF0E0EE55FC4F678527
:100A800089E70E9424056C2F8DE30E9424056C2FBA
:100A900082E40E942405CF91089586E20E941E05FB
:100AA0000895CF93DF93EC016C818CE10E942405C3
:100AB0006D818DE10E9424056E818EE10E942405E6
:100AC0006F8180E20E942405688581E20E942405EE
:100AD000698582E20E9424056A8583E20E942405DA
:100AE0006B8584E20E9424056C8585E20E942405C2
:100AF0006D858AE20E9424056E858EE60E9424059B
:100B00006F858FE60E942405688980E70E9424058E
:100B1000698981E70E9424056A8982E70E94240589
:100B2000DF91CF910895CF92DF92EF92FF92CF9312
:100B3000DF936B017C01C11488E3D8068CE9E806D9
:100B40008CE1F80628F5C701B60120E836E948E946
:100B500050E00E94D725E901689760E879E687E6CA
:100B60009FEF0E94B3256C0D7D1D8E1D9F1DF2E031
:100B7000660F771F881F991FFA95D1F721E732E09A
:100B800040E050E00E94D725F22EE32E80E421C001
:100B9000C701B60120E03DE241E351E00E94D725C4
:100BA000E901689760E073ED8EEC9EEF0E94B3253B
:100BB0006C0D7D1D8E1D9F1D660F771F881F991F51
:100BC00021E732E040E050E00E94D725F22EE32EEC
:100BD00080E66C2F6F71680F85E70E9424056E2DEB
:100BE00086E70E9424056F2D87E70E942405DF9188
:100BF000CF91FF90EF90DF90CF900895682F8DE612
:100C00000E94240508958F929F92AF92BF92CF9237
:100C1000DF92EF92FF92CF93DF93D82F83E00E9471
:100C20001E0580939D0384E00E941E0580939C0313
:100C300060E086E00E94240561E087E00E942405D0
:100C40006FE789E00E94240565E08AE00E942405A0
:100C500065E18BE00E94240562E18CE00E9424059E
:100C60006DEF8DE00E94240560E08EE00E94240577
:100C7000DD2319F08BE291E008C02091C90333E134
:100C8000239FC0011124825C9E4F0E9451056CE895
:100C900080E30E9424056FE082E30E94240562E461
:100CA00083E30E9424058091CA0387FF02C064E1A8
:100CB00001C06AE084E30E9424056AE285E30E94A1
:100CC00024056DE286E30E94240564ED87E30E941B
:100CD000240560E088E30E94240560E089E30E9427
:100CE0002405D11109C0C090AB03D090AC03E090B3
:100CF000AD03F090AE0307C0C5E9CC2EC1ECDC2EED
:100D0000ED2CCEEDFC2ECAE38F2C9924AA24BB2413
:100D1000682D8C2F0E942405682D85E08C0F0E9481
:100D20002405FE2CED2CDC2CCC24CF5FCE3361F7D8
:100D30006FEF83E40E9424056FEF84E40E94240592
:100D40006FEF85E40E9424056FEF86E40E9424057E
:100D5000DD2311F066E002C06091AF038DE60E94D2
:100D6000240560E089E70E9424056091B0038AE7CA
:100D70000E94240560E083E70E94240560E084E788
:100D80000E942405D11109C06091A7037091A803A6
:100D90008091A9039091AA0304C060EC7AEC89E8E1
:100DA00096E30E949305DF91CF91FF90EF90DF9043
:100DB000CF90BF90AF909F908F90089561E087E0B3
:100DC0000E94240564E28EE70E94240563E088E027
:100DD0000E94240560E088E00E94240565E087E029
:100DE0000E94240562E085E00E94240583E00E94C1
:100DF0001E0580939D0384E00E941E0580939C0342
:100E0000089583E00E941E0580939D0384E00E9464
:100E10001E0580939C0361E087E00E9424056AE040
:100E200070E080E090E00E94331B0E94DE0600002C
:100E30000895CF92DF92FF920F931F93CF93DF938A
:100E40001F92CDB7DEB7082F162F8EE399830E942D
:100E50002405F02EC02E9981D92E8C2D8F19811743
:100E600038F4F60161916F018FE70E942405F5CFF8
:100E700064E085E00E94240583E00E941E058093C3
:100E80009D0384E00E941E0580939C030E94101B1A
:100E9000609398037093990380939A0390939B03B4
:100EA00069E087E00E94240581E080939F030F9012
:100EB000DF91CF911F910F91FF90DF90CF90089518
:100EC0000F931F930E94190780919F03813099F41B
:100ED0000E94101B009198031091990320919A038E
:100EE00030919B03601B710B820B930B603A764829
:100EF0008140910548F380919F03813031F467EA86
:100F000071E08AE094E00E94181E1F910F910895ED
:100F10000F931F9380919F03823021F410929F03BF
:100F200081E020C080919F038130D9F40E94101B82
:100F3000009198031091990320919A0330919B039B
:100F4000601B710B820B930B613A764881409105CF
:100F500040F061E087E00E94240510929F0382E048
:100F600001C080E01F910F910895CF93DF93EC01B2
:100F70004AE050E06D2F70E08AE094E00E94DD1EB0
:100F80006EE28AE094E00E94EA1DBE0184E076955C
:100F900067958A95E1F76F7077274AE050E08AE01D
:100FA00094E00E94DD1E6EE28AE094E00E94EA1D59
:100FB000BE016F7077274AE050E08AE094E00E941B
:100FC000DD1EDF91CF910895D82FC0E0CD1780F4BA
:100FD0005F9A64E670E080E090E00E94331B5F98C7
:100FE00064E670E080E090E00E94331BCF5FEECFBC
:100FF0006CE271E080E090E00E94331BE6CF0F933B
:101000001F93CF93DF93EC01062F15E0115051F0A1
:10101000CE010E94C626081741F0602FCE010E9423
:10102000CE26F4CF82E00E94E407DF91CF911F919A
:101030000F910895A0E0B0E0E0E2F8E00C941A26E9
:10104000482E562EC0E0D0E0612C712CE12CF12C02
:1010500000E010E041100CC06090000486E4689E3F
:101060003001112459E1E52EF12C06EE13E01EC0EB
:1010700091E049120FC060900004E6E46E9E3001DA
:101080001124FBE16F0E711C49E2E42EF12C02EAFF
:1010900013E00CC082E0481209C028E1622E7724D8
:1010A0007394EE24E394F12C0FEF13E043018C0EC4
:1010B0009D1E1092A1031092A0033401A62CA81823
:1010C000B12CC30101966C01AE14BF04A8F4A00EAC
:1010D000B11E511006C0C3010E94C626F5018083CF
:1010E00005C0F5016081C3010E94FF07F501808101
:1010F0000E94D1013601E2CFC301511018C0C301D3
:101100000E94C626B82EC6010E94C6262B2D30E0AE
:10111000322F2227282B8091A0039091A1038217C0
:10112000930779F4C0E0D0E05524539493CF36016F
:101130006091A1030E94FF076091A003C6010E9475
:10114000FF07C05EDE4FC13E92E0D90708F482CFB0
:10115000852DCDB7DEB7E0E10C94362661E082E064
:101160000E941A08089560E082E00E941A088091A7
:10117000FF03853020F01092FF030E94AE0880919B
:10118000FF0380930004089561E080E00E941A0844
:1011900061E081E00E941A08089560E080E00E940A
:1011A0001A08882351F060E081E00E941A08882321
:1011B00021F08091A203883349F00E942F020E94FF
:1011C000EA0181E00E944F020E94C4080895CF9373
:1011D000C82F0E94101B60935C0370935D03809383
:1011E0005E0390935F03C0937103CC2329F040E02A
:1011F00051EE60E070E004C040E855E260E070E06D
:101200008CE594E00E944320CF9108959091600373
:10121000492F4F7050E0BA016F5F7F4F292F30E0A8
:10122000E4E035952795EA95E1F76217730759F0E1
:10123000FA01EF59FC4F808381E0890F8F70907F16
:10124000892B8093600308956EE770E08CE594E04D
:101250000E94C9010895A3E1B1E0E1E3F9E00C9433
:101260001B26E1EBF3E0712C8191882321F073942C
:1012700028E17212F9CF63EB71E08AE094E00E94FA
:10128000181E4AE050E0672D8AE094E00E94E41EB8
:1012900080E00E9403060E94DE068E010E5F1F4F53
:1012A000C12CD12C7601C39466246A945C2C0E94D4
:1012B000041B4B015C012091B00330E0A0E1B7E2D8
:1012C0000E9491259B01AC01C701B6010E94B32584
:1012D0002091A7033091A8034091A9035091AA033C
:1012E000620F731F841F951F2091E7033091E8035D
:1012F0004091E9035091EA03261737074807590739
:1013000018F4F801608225C08C2D0E94370561E039
:1013100070E080E090E00E94331BF80110820E9490
:10132000041B681979098A099B09643F714081058A
:10133000910540F40E944D05F8019081981778F7C7
:101340008083EDCF50FE03C046985F9A02C0469A54
:101350005F982FEFC21AD20AE20AF20A0F5F1F4FFC
:101360008FEFC816D104E104F10409F09FCFCE013C
:101370009395FC01D82E7FEF68EC2E2F281B2715A4
:1013800010F051E056C0DE01129651E02FEF41E01F
:101390003D91321710F0322F01C0452F5F5F5F3F44
:1013A00011F0232FF5CF4193242F30E0A1E0B0E0DE
:1013B000AC0FBD1FA20FB31F5C93413079F0DE016B
:1013C000A20FB31F5C93423049F0AFEFBFEFAC0FF9
:1013D000BD1FA20FB31F6C934E3F78F6A2E0B0E0A2
:1013E000AC0FBD1FA20FB31F7C934D3F30F6A3E09F
:1013F000B0E0AC0FBD1FA20FB31F6C93BECF452F43
:10140000242F30E0FC01E20FF31F6081AFEFB0E06A
:10141000AC0FBD1FA20FB31F2C91621748F44150AF
:10142000DC01A40FB11D2C9120836C934111E8CFF6
:101430005F5F571520F3372D369520E0231770F4A2
:10144000DC01A20FB11D4C91522F530FFC01E50F8F
:10145000F11D50815C9340832E5FF0CFF1EBEF2EB6
:10146000F3E0FF2E8C01802F8D19871598F4F80179
:10147000C1908F014AE050E06C2D8AE094E00E9418
:10148000D51E6CE28AE094E00E94EA1DF701C19249
:101490007F01E9CF8AE094E00E94F21D81E0CD5EF9
:1014A000DE4FEFE00C9437261F920F920FB60F928B
:1014B00011241F932F933F934F935F936F937F93C9
:1014C0008F939F93AF93BF93CF93DF93EF93FF934C
:1014D000C0918600D09187008091170390911803E6
:1014E00020913903211155C09E01281B390B809191
:1014F000EB039091EC03A091ED03B091EE0385FD19
:1015000002C036952795253C49E03407B8F1409153
:101510000A0150E060E070E02CE1B695A795979540
:1015200087952A95D1F70097A105B10521F481E0AF
:1015300090E0A0E0B0E084179507A607B707D8F4BD
:1015400080910A018F3FB9F040E080910A0148176D
:1015500080F4842F90E0880F991FFC01E75EFC4F18
:1015600020813181FC01E55FFE4F318320834F5F95
:10157000ECCF10923A0310920A010BC02D3B82E08F
:10158000380720F080910A018031D8F08FEF8093E6
:101590000A01D0931803C0931703FF91EF91DF91D5
:1015A000CF91BF91AF919F918F917F916F915F91FB
:1015B0004F913F912F911F910F900FBE0F901F9051
:1015C000189510910A0181E0810F80930A01C901E9
:1015D0000E946204E12FF0E0EE0FFF1FE75EFC4F78
:1015E00091838083D6CF83E0809380008AE98093C3
:1015F00081008091EB0386FD05C0809181008064AD
:10160000809381008FEF9FEF9093890080938800F3
:1016100080916F00806280936F000895CF93DF9375
:101620000E94B30880910004843039F582E00E9462
:10163000541CC1E0D0E0892B11F4C0E0D0E083E07D
:101640000E94541C892B19F082E090E002C080E0D7
:1016500090E08C2B9D2B8230910539F083309105E1
:1016600039F0019739F481E006C01092000405C0FA
:1016700082E001C083E080930004DF91CF91089560
:101680006F3018F086958058089589E0689F802D06
:1016900011240895A0E0B0E0E0E5FBE00C942226E0
:1016A000C82F0E94101B0091C8021091C9022091FE
:1016B000CA023091CB026B017C01C01AD10AE20A46
:1016C000F30A9701860149E8C41643E1D406E10410
:1016D000F10410F01092CC026093C8027093C9021A
:1016E0008093CA029093CB02209139038FEF820F2F
:1016F0008230E8F5E091CC02EE2309F46EC1E130CE
:1017000011F482E0D8C1E03178F581E08E0F80934A
:10171000CC02F0E0E75EFC4FC083803109F0D4C119
:10172000EBE1F3E0213029F4A181A695A695808113
:1017300008C080819181A92FA695A695A69596951A
:101740008795A03148F4B0E090E0AA0FBB1FA55FD9
:10175000BE4F11969C938E9310923A03329683E07B
:10176000E932F807F9F6B0C11092CC02ADC12330CE
:1017700009F023C1E091CC02E11118C0CF3009F08B
:1017800011C10E94041B009147031091480320914E
:10179000490330914A03601B710B820B930B62303B
:1017A00071058105910508F089C1FCC0E73148F455
:1017B00081E08E0F8093CC02F0E0E85EFC4FC083A6
:1017C000F1C0E73109F0ECC0C111EAC040E050E0DF
:1017D000ABE0CA01B3E0880F991FBA95E1F7A49F67
:1017E0009001A59F300D1124F901E75EFC4F608147
:1017F000E1817E2F777075956795FC01EE0FFF1FD5
:10180000E55FFE4F71836083F901E65EFC4FB081B6
:10181000B695B695B695E181FE2FF295FF0FF07E55
:101820006F2F6B2BE695E695E6957E2F7770759575
:101830006795FC01EE0FFF1FE35FFE4F718360832E
:10184000F901E55EFC4FB081B295B695B695B370DF
:10185000C181DC2FDD0FDD0F6D2F6B2BC295C6957F
:10186000C695C370E281E170EE0FEE0F7E2F7C2BE8
:1018700075956795FC01EE0FFF1FE15FFE4F7183C9
:101880006083F901E35EFC4FB081B695E181FE2FE4
:10189000F795FF27F7956F2F6B2BE6957E2F7770C7
:1018A00075956795FC01EE0FFF1FEF5EFE4F71838C
:1018B0006083F901E25EFC4FB081B295BF70E181B7
:1018C000FE2FF295F07F6F2F6B2BE295EF707E2F3E
:1018D000777075956795FC01EE0FFF1FED5EFE4F6B
:1018E00071836083F901E15EFC4FB081BB1FBB27B0
:1018F000BB1FC181DC2FDD0F6D2F6B2BCC1FCC27C5
:10190000CC1FE281E370EE0F7E2F7C2B75956795DF
:10191000FC01EE0FFF1FEB5EFE4F71836083F90148
:10192000EF5DFC4FB081B695B695E181FE2FF29543
:10193000FF0FFF0FF07C6F2F6B2BE695E6957E2F48
:10194000777075956795FC01EE0FFF1FE95EFE4FFE
:1019500071836083F901EE5DFC4F2081229526950D
:1019600027703181E32FEE0FEE0FEE0F6E2F622BFB
:10197000732F72957695777075956795FC01EE0FCC
:10198000FF1FE75EFE4F718360834F5F5F4F423002
:10199000510509F01ECF80912F0383FF10923A0367
:1019A0001092CC020E94041B60934703709348037B
:1019B0008093490390934A0387C0243009F084C080
:1019C0006091CC0261110BC0C83AB1F41092A1032E
:1019D0001092A00388EA0E94D10181E06CC06130BE
:1019E00019F4C093C70204C0623031F4C093C60238
:1019F0008C2F0E94D1015AC0E091C6022E2F30E0F8
:101A0000220F331F462F50E0C90102968417950715
:101A10003CF0633268F7FA01EA5EFC4FC083E8CF1E
:101A20002D5F3F4F8C2F90E06091A0037091A10338
:101A30004217530749F4982F8827862797279093B2
:101A4000A1038093A00332C06817790769F58091DC
:101A5000C702813049F5E13118F080E18093C60278
:101A6000F090C602CAE1D3E000E010E00F15D0F418
:101A7000FE013197808190E0982F88272881822B62
:101A800063E0969587956A95E1F70E946204F801F4
:101A9000EE0FFF1FE55FFE4F918380830F5F1F4FA7
:101AA0002296E4CF10923A031092CC028091CC029D
:101AB000882351F08F5F8093CC0206C08091CC02C6
:101AC0008F5F8093CC026ECFCDB7DEB7E8E00C9489
:101AD0003E26CF93DF93E82FF0E0EA51FC4FE185FB
:101AE000E03150F4F894F0E0EE0FFF1FE55FFE4F99
:101AF0008081918178945FC08EE08E0F8B3058F496
:101B0000F0E0E25FF10924E62E9FC0012F9F900DC7
:101B100011240C9650C0E03F09F448C038F4E1317C
:101B2000A1F0E231A1F0E03139F409C0ED3FC1F19B
:101B3000EE3FC9F1E13F89F180E092E03CC082E0F4
:101B40000E94541C892B19F134C083E0F9CF82E044
:101B50000E94541CC1E0D0E0892B11F4C0E0D0E019
:101B600083E00E94541C892B19F082E090E002C0AF
:101B700080E090E08C2B9D2B8230910541F08330EA
:101B8000910541F00197A9F086EA92E014C08CE03B
:101B900090E011C089E591E00EC086E090E00BC0B6
:101BA0008AEF93E008C08FEF93E005C080E090E0FB
:101BB00002C084EF93E0DF91CF910895A2E2B0E0FC
:101BC000E4EEFDE00C9418269E012F5F3F4F80E16C
:101BD000D9011D928A95E9F761EE71E08AE094E0FF
:101BE00029A33AA30E94181E0E9401071D8A1E8A7B
:101BF0001F8A188E312C212C00E0812C912C54014D
:101C000070EC472E7DE9572E78E5672E75E3772E29
:101C1000E0E5CE2EE3ECDE2EE12CF12C84EF91E01A
:101C2000A0E0B0E08D8F9E8FAF8FB8A380EC97EFD0
:101C3000AAEBB7E3898F9A8FAB8FBC8F80EC9DE9BD
:101C4000A8E5B5E3898B9A8BAB8BBC8B8AE094E0DB
:101C50000E947D1C892B09F4E1C08AE094E00E9477
:101C6000A11C9C0133272C32310509F442C0ACF48D
:101C70002332310509F0ABC019821A821B821C8203
:101C80001D821E821F82188619861A861B861C8654
:101C90001D861E861F86188A60C02434310529F0EF
:101CA0002335310509F4B2C092C064E48AE094E0BF
:101CB0000E94EA1D2AE030E040EC5DE968E575E34A
:101CC0008AE094E00E94781E6CE28AE094E00E9430
:101CD000EA1D2AE030E040EC57EF6AEB77E38AE058
:101CE00094E00E94781E6CE28AE094E00E942A1E32
:101CF000ADCF0F5F043009F0A9CF29813A814B8124
:101D00005C81A8EEB3E00E94A025698B7A8B8B8B57
:101D10009C8B2D813E814F8158850E94A025698F23
:101D20007A8F8B8F9C8F29853A854B855C852D8F8B
:101D30003E8F4F8F58A32D853E854F8558890E9431
:101D4000A0256B017C0160323EE47307810591059B
:101D500030F462E38CE10E94240500E077CF603329
:101D600045E774078105910510F462E2F3CF603412
:101D70005CE975078105910510F466E2EBCF80E51B
:101D8000C81683ECD806E104F10410F462E1E2CF56
:101D900090E6C9169AEED906E104F10410F465E163
:101DA000D9CFA0E7CA16A1E1DA06A1E0EA06F1045C
:101DB00010F461E0CFCFB0EACB16B6E8DB06B1E0B5
:101DC000EB06F10410F463E0C5CF65E0C3CF10ED7E
:101DD000180F1A3008F03ACFE1E0F0E0EC0FFD1FE9
:101DE00024E0029FE00DF11D112420813181428108
:101DF0005381AAE0B0E00E94A025610F711D811DF2
:101E0000911D608371838283938320CF49885A8890
:101E10006B887C88812C912C540118CF81149104FB
:101E2000A104B10489F4C301B2010E94930561E0E9
:101E300070E080E090E00E94331B1D8A1E8A1F8A9A
:101E4000188E312C22242A948D8D9E8DAF8DB8A1B1
:101E500088169906AA06BB06D0F40E944D052D8966
:101E60003E894F89588D280F311D411D511D2D8BE5
:101E70003E8B4F8B588F381608F4382E821508F495
:101E8000282E3FEF831A930AA30AB30A56C0C30150
:101E9000B20128EE33E040E050E00E94D725BA01BD
:101EA000A9012AE030E08AE094E00E94C61E6CE2BC
:101EB0008AE094E00E94EA1D4AE050E0632D8AE047
:101EC00094E00E94D51E6CE28AE094E00E94EA1D34
:101ED0006D897E898F89988DA50194010E94D725EF
:101EE000BA01A9012AE030E08AE094E00E94C61E0F
:101EF0006CE28AE094E00E94EA1D4AE050E0622D24
:101F00008AE094E00E94D51E6CE28AE094E00E9490
:101F10002A1E4C0C5D1C6E1C7F1C898D9A8DAB8D0E
:101F2000BC8D84159505A605B70520F449885A8807
:101F30006B887C88812C912C540129893A894B89A2
:101F40005C89283E33404105510509F07FCEA296B9
:101F5000E2E10C943426ACE1B0E0E1EBFFE00C945C
:101F600022260E94101B6B017C0181E00E94030667
:101F700014E703E0198361E0CE0101960E94600737
:101F800000939F030E94DE066AEF70E080E090E01D
:101F90000E94331B80919F03833089F48AE094E090
:101FA0000E947D1C892B59F40E94101B6C197D091D
:101FB0008E099F096038734C894C9140D8F280910A
:101FC0009F03833009F44FC08FE70E94FC040E94F6
:101FD0000F058983843511F083E05CC00E940F05F2
:101FE00010927203809373030E940F052091720375
:101FF00030917303280F311D3093730320937203C4
:102000000E940F05809374030E940F05809375034F
:10201000813110F7F12C0F2D10E08091750390E0C5
:10202000880F991F0817190740F40E940F05F8013F
:10203000EA58FC4F8083F394EECF80E7898361E018
:10204000CE0101960E94600783E080939F030E9467
:10205000DE0662E370E080E090E00E94331B809136
:102060009F03833011F482E015C08FE70E94FC04C7
:102070000E940F058983803509F0AECF0BEC13E089
:102080000E940F05F80181938F01F3E0063E1F07C0
:10209000B9F781E06C96E8E00C943E26CF93C82F08
:1020A000682F8AE094E00E94EE1C909196039C2792
:1020B00090939603CF910895A1E0B0E0E2E6F0E1BD
:1020C0000C94282699830E944E109981892F0E9492
:1020D0004E102196E2E00C9444261F93CF93DF9399
:1020E000182FEB011092960365EB8AE094E00E94B2
:1020F000EE1C62E68AE094E00E94EE1C812F0E94B2
:102100004E10CE010E945C10DF91CF911F91089577
:10211000609196038AE094E00E94EE1C0895A1E28B
:10212000B0E0E5E9F0E10C9424267B018A018C30D3
:1021300009F453C108F040C0863009F4BCC018F55A
:10214000833009F491C070F4813009F472C0823098
:1021500009F04AC26BE170E082E00E946D100BEC66
:1021600013E078C0843009F487C0853009F03CC2A0
:102170006091750370E0660F771F85E00E946D1017
:1021800006E713E086C0893009F4A7C070F48730F1
:1021900009F49BC0883009F027C261E070E088E054
:1021A0000E946D108091000425C28A3009F4CAC0D3
:1021B0008B3009F4F2C018C28A3609F475C1D8F41C
:1021C000873609F43AC138F4853609F40EC18636EB
:1021D00009F41FC109C2883609F437C1893609F0EC
:1021E00003C261E070E089E60E946D100E94EA017E
:1021F0000E942F02F7C18D3609F4D4C138F48B3612
:1022000009F491C18C3609F49AC1EEC18E3609F4F5
:10221000DEC1873C09F0E8C161E070E087EC0E9414
:102220006D1081E00E944E100E948810109297035A
:10223000E5C169E270E081E00E946D1002EA13E0FE
:10224000F80181918F010E944E10F3E00B3C1F07B3
:10225000B9F7D2C1F80181918F010E944E10F3E0CD
:10226000063E1F07B9F7C8C161E070E083E00E9435
:102270006D100E94AB0FBEC161E070E084E00E946F
:102280006D1081E00E944E100E9488100E94DE0DA9
:10229000B5C18091750390E0880F991F980126576A
:1022A00033402817390708F0A7C1F80181918F0141
:1022B0000E944E10EECF62E070E086E00E946D104A
:1022C00086E893E00E945C1097C161E070E087E0CF
:1022D0000E946D10809174038DC186E6898361E050
:1022E000CE0101960E9460070E94DE0683E0809383
:1022F0009F0368EC70E080E090E00E94331B8091C7
:102300009F038430D9F48FE70E94FC040E940F05DC
:102310008983863469F460E270E089E00E946D1080
:1023200010E20E940F050E944E101150D1F764C1B7
:1023300061E070E089E00E946D1054C161E070E0DE
:1023400089E055C169E170E08AE00E946D1082E089
:102350008093E60320919E038091EB039091EC0320
:10236000A091ED03B091EE03222311F0806801C02B
:102370008F778093EB039093EC03A093ED03B093DE
:10238000EE0306EE13E0F80181918F010E944E10DA
:10239000F3E00F3F1F07B9F72FC161E270E08BE058
:1023A0000E946D1080913A038F3F39F080913A037B
:1023B00091E0980F90933A0302C080913A030E94F3
:1023C0004E1010E0812F0E94690D0E948D040E9422
:1023D0005C101F5F1031B1F70FC161E070E08CE05D
:1023E0000E946D108091FF0305C161E070E085E6F9
:1023F0000E946D1089E2E816F10409F0FAC0D801D4
:10240000E2EAF3E08D91819383E0EB3CF807D1F7AA
:10241000E9C061E070E086E60E946D10EBE1EE1627
:10242000F10409F0E6C0D801EBECF3E08D91819363
:1024300083E0E63EF807D1F7D5C061E070E087E6BB
:102440000E946D100E94C408CDC061E070E088E673
:102450000E946D1085E789838BE1EBECF3E0DE01F0
:10246000129601900D928A95E1F76CE1CE010196EA
:102470000E9460070E94DE0683E080939F0360E273
:1024800073E080E090E00E94331B80919F038430D2
:1024900009F0AFC08FE70E94FC040E940F058983FA
:1024A000853509F0A6C09EC061E070E08AE60E9412
:1024B0006D1089E6898361E0CE0101960E94600774
:1024C0000E94DE0683E080939F0360E273E080E079
:1024D00090E00E94331B80919F03843009F089C0F3
:1024E0008FE70E94FC040E940F0589838E010E5F16
:1024F0001F4F7E01EDE1EE0EF11C0E940F05F80169
:1025000081938F01EE15FF05C1F78BE1FE01329635
:10251000ABECB3E001900D928A95E1F789818934A3
:1025200009F067C05FC061E070E08BE60E946D104B
:10253000F8018081809300040E94CD0853C061E0BF
:1025400070E08CE60E946D10F0E2EF16F10461F489
:1025500087E6898380E2F801DE01129601900D92F0
:102560008A95E1F761E203C087E4898361E0CE01E7
:1025700001960E9460070E94DE0683E080939F031D
:102580006CE474E080E090E00E94331B80919F0334
:10259000843079F58FE70E94FC040E940F05873490
:1025A00041F520C061E070E08DE60E946D1089E188
:1025B000E816F104F1F4D801E6EEF3E08D91819391
:1025C00083E0EF3FF807D1F70E94F30A0BC061E008
:1025D00070E08EE60E946D10F80180818093FF0309
:1025E0000E94AE0881E006C061E070E08AEC0E94C3
:1025F0006D1080E00E944E100E948810A196E6E0C7
:102600000C944026A0E0B0E0E8E0F3E10C94222630
:10261000CAE5D2E014E606E035E0F32E44E0E42E0D
:1026200053E0D52E62E0C62E8AE094E00E947D1C25
:10263000892B09F49BC08AE094E00E94A11C282FFA
:102640008093C5024091C40250E04730510560F7C5
:10265000FA01EA5AFF4F0C944F26853B29F781E097
:102660008093C402E1CF823609F07DC0C092C402DB
:10267000DBCF8093C3028093C202D092C402D4CF36
:102680009C0133273093C1022093C0029091C20273
:1026900098279093C202E092C402C6CF382F222717
:1026A0004091C0025091C102242B352B3093C102BE
:1026B0002093C0029091C20298279093C202F09298
:1026C000C4022536310508F4AFCF61E070E08CEC30
:1026D0000E946D1081E00E944E100E94881043C03D
:1026E0002091BE023091BF02F901E65AFD4F80836E
:1026F0009091C20298279093C202C90101969093CB
:10270000BF028093BE022091C0023091C1028217A5
:10271000930708F489CF0093C40286CF8091C20248
:1027200082130BC06091BE027091BF024AE552E075
:102730008091C3020E948F100DC062E070E08BECAC
:102740000E946D108091C3020E944E1080919603EA
:102750000E944E10FE01812F11928A95E9F7109286
:10276000BF021092BE021092C4025ECFCDB7DEB798
:10277000E8E00C943E2681E08093970380919703D4
:10278000882349F08AE094E00E947D1C892BB1F3F4
:102790000E940213F3CF0895AAE2B0E0E2EDF3E164
:1027A0000C9420260E94041B6B017C0181E00E9496
:1027B00003068AE094E00E947D1C892B29F08AE0C0
:1027C00094E00E94A11CF5CF5F9811E072E6B72E4D
:1027D000E9E2AE2E03E00E94041B6C197D098E090C
:1027E0009F09693C710581059105D0F11123C1F163
:1027F0000E94041B6B017C01469A80ED97E00E94C9
:10280000FF02B982E2EAF3E0DE0112968A2D01901E
:102810000D928A95E1F76AE2CE0101960E94600767
:10282000469880E090E00E94FF0200939F030E9480
:10283000DE0662E370E080E090E00E94331B80914E
:102840009F03843061F400939F038FE70E94FC0490
:102850000E940F0511E0823419F410E001C011E06C
:1028600082E10E94541C892B81F411E00EC05F9A12
:10287000469A8AE094E00E94A11C8D309105A9F04F
:102880005CF40A9791F05F9846988AE094E00E9481
:102890007D1C892B61F79FCF8332910569F08234CB
:1028A000910589F70E94BB13EECF66ED70E08AE0D8
:1028B00094E00E94061EE7CF0E94DE0DE4CF8F92C7
:1028C0009F92AF92BF92CF92DF92EF92FF921F93AF
:1028D000CF93DF9382E10E94541C892B09F089C0B9
:1028E00068EC70E080E090E00E94331B80E090E0B4
:1028F0000E94FF020E94041B4B015C016B017C01E2
:1029000080ECC80E82E1D81EE11CF11C0E94041B61
:102910006C157D058E059F0530F482E10E94541CE4
:10292000892BA1F364C082E10E94541C892B09F019
:102930005EC080ED97E00E94FF020E94041B6B01C5
:102940007C01D0E0C1E088E4880E86E2981EA11CDC
:10295000B11C11E082E10E94541C892B21F58C14DA
:102960009D04AE04BF0430F480ED97E00E94FF02A6
:10297000D1E0F0CF0E94041B6C197D098E099F09DC
:10298000693C71058105910528F30E94041B6B01C8
:102990007C01C12719F080ED97E002C080E090E053
:1029A0000E94FF02D7CF80E090E00E94FF02DD236B
:1029B000B9F08091FF0390E0019665E070E00E941D
:1029C000C3258093FF030E94AE080E940E0B0E9455
:1029D000CD0864EF71E080E090E00E94331B09C0F5
:1029E00080E00E944F020E942B090E94C4080E94AE
:1029F000CC13DF91CF911F91FF90EF90DF90CF909C
:102A0000BF90AF909F908F900895CF92DF92EF92FA
:102A1000FF9280E00E945C030E94200361E086E058
:102A20000E94E81B61E085E00E94E81B60E082E113
:102A30000E94E81B60E082E00E94E81B61E082E007
:102A40000E94211C60E083E00E94E81B61E083E0BB
:102A50000E94211C60E084E00E94E81B61E084E0A9
:102A60000E94211C0E94F30260E070E08AE094E082
:102A70000E94731D0E940E0B0E94CD080E94F30A53
:102A80008FEF80933A030E942C0378940E94041BDA
:102A90006B017C0180913A038F3F59F40E94041B23
:102AA0006C197D098E099F09603D7740810591056C
:102AB00088F380ED97E00E94FF0261E082E10E94CE
:102AC000211C5F9A8AE094E00E947D1C892B29F0EA
:102AD0008AE094E00E94A11CF5CF6EEE71E08AE0DE
:102AE00094E00E94E71D86E893E00E94B50765E048
:102AF00072E08AE094E00E94E71D4AE050E066E060
:102B000070E08AE094E00E94AE1E62E370E080E034
:102B100090E00E94331B8AE094E00E947D1C0497A1
:102B20000CF18AE094E00E94A11C82349105D1F45A
:102B30008AE094E00E94A11C8E34910599F48AE009
:102B400094E00E94A11C8434910561F48AE094E031
:102B50000E94A11C819731F480E090E00E94FF0266
:102B60000E94CC134091A3035091A4036091A5034C
:102B70007091A603DB01CA010197A109B10904976D
:102B8000A105B10568F440933903433029F440EAC4
:102B900056E861E070E004C040E052EC61E070E0B3
:102BA0008CE594E00E9443200E945F145F9880E0CF
:102BB00090E00E94FF020E94F30A10925903809154
:102BC000EB0383FF11C08091B703882351F08091FC
:102BD000BE03882331F08091C503882311F087E07C
:102BE00001C085E08093590380E00E940306809134
:102BF0005A030E9437050E94DE061092CF021092FF
:102C0000CE021092CD02F12C809100048F15B0F00D
:102C100062E370E080E090E00E94331B80ED97E07B
:102C20000E94FF0262E370E080E090E00E94331BAC
:102C300080E090E00E94FF02F394E6CF8091CA0307
:102C400084FF08C0982F987181E0983109F080E0E6
:102C50000E94E7088FE00E945C03FF90EF90DF90F6
:102C6000CF900895EF92FF920F931F93CF93DF932E
:102C70008C016EE770E08CE594E00E94C901E801E8
:102C8000F12CF0E2EF2E8E0188818D57823048F4CE
:102C90006DE770E08CE594E00E94C90188818E2583
:102CA00088832196F80160818CE594E00E94551F8D
:102CB000F394F9E0FF12E7CF6EE770E08CE594E063
:102CC0000E94C901CDB7DEB7E6E00C944026A9E02A
:102CD000B0E0EDE6F6E10C94282690915B039111AB
:102CE0000EC09EEF99838A836B8350E0559547957C
:102CF0004C832D83198618861F821E822EC0409118
:102D00006003842F90E0B4E095958795BA95E1F73C
:102D1000242F2F7030E08217930719F18DEF8983EC
:102D20001B82FE01349650E0842F90E0A4E095953C
:102D30008795AA95E1F7242F2F7030E0821793072B
:102D400049F0DC01AF59BC4F8C918193405F5F5FCC
:102D5000563051F7409360035A83CE0101960E948A
:102D6000321680915B0390E0019666E070E00E946D
:102D7000C32580935B032996E2E00C944426A0E0EF
:102D8000B0E0E5ECF6E10C9421266C016EE770E012
:102D90008CE594E00E94C9018601E12CF12CC0E091
:102DA000D0E030E2B32EF801608183E8860F8230F4
:102DB00078F46DE770E08CE594E00E94C901F801B9
:102DC00060816B2570E08CE594E00E94C90104C02D
:102DD0008CE594E00E94551FE114F10459F0F801CC
:102DE00080819E01280F311DC901C92FDD27C80F21
:102DF000D91FDD273FEFE31AF30A89E0E816F10453
:102E000059F028E0E216F10421F48C2F8095F601A8
:102E100080870F5F1F4FC7CFCDB7DEB7E9E00C94B7
:102E20003D26A9E0B0E0E7E1F7E10C942826E82F81
:102E3000362F80915B0390E0019664E270E00E947F
:102E4000C32580935B0358E9598350E15A8381304D
:102E500089F048F08230B9F08330D9F48B8381EF68
:102E60008C833D8319C085E08B8381EF8C832F5F3A
:102E70002D8312C08B8381EF8C8384E6489FA00151
:102E800011245D8309C084E08B8381EF8C83ED8303
:102E900003C00E94240904C0CE0101960E94BF16FF
:102EA0002996E2E00C944426A2E0B0E0EAE5F7E1DE
:102EB0000C941D26182F762E2A8349830E94101BFE
:102EC0006B017C018091710380905C0390905D03A5
:102ED000A0905E03B0905F032A8149818823C1F0EE
:102EE000D701C60188199909AA09BB094C015D01DE
:102EF00091EE89169EE29906A104B10420F12417EF
:102F000008F4422F202F672D812F0E94111713C024
:102F1000D701C60188199909AA09BB094C015D01AD
:102F200091E3891695E79906A104B10460F0672D35
:102F3000812F0E946716C0925C03D0925D03E092DD
:102F40005E03F0925F032296EDE00C943926A2E234
:102F5000B0E0EDEAF7E10C941E268CE00E941E051D
:102F600081110DC06DE072E08AE094E00E94181EAD
:102F70005F9A80E00E9403060E94DE065F988CE55F
:102F800094E00E94FB1E892B01F18CE594E00E94E5
:102F9000281F90913903992319F00E944A0BEFCF13
:102FA0004091CE0250E09A012F5F3F4F2F7133279F
:102FB0006091CF0270E02617370709F3FA01E75254
:102FC000FD4F80832093CE02DACF809139038111A7
:102FD00006C080919F03843009F094C00DC08AE040
:102FE00094E00E947D1C892BA1F38AE094E00E946A
:102FF000A11C0E944A0BF3CF0E94101B61157105A2
:103000008105910549F060934B0370934C038093C5
:103010004D0390934E030CC081E090E0A0E0B0E03F
:1030200080934B0390934C03A0934D03B0934E03B6
:1030300080913D0390913E03816090933E03809385
:103040003D0383E080939F038FE70E94FC0409EF18
:1030500012E00E940F05F80181938F01F3E0023026
:103060001F07B9F7209102038091F902982F922748
:1030700096FF3BC090E4922790930203982F987399
:103080009833F1F410E0212F30E08091F90287703D
:1030900090E0821793074CF11F5F2091CA03812FA4
:1030A00090E0FC01E750FD4F24FF04C080810E94A6
:1030B0000609E9CF60818CE594E00E94551FE3CFBB
:1030C0008F7399F48091FA02809346038091FB02FA
:1030D000809344038091FC02809343038091FF021C
:1030E00090E090933C0380933B038091CD0281302C
:1030F00019F482E08093CD028091CD02833011F4E7
:103100001092CD020E94101B6B017C0180913F0345
:1031100090914003A0914103B09142030097A10513
:10312000B105C9F0A7019601281B390B4A0B5B0BAF
:10313000DA01C901883B9B40A105B10560F00E94FE
:103140004D058093450310923F0310924003109267
:1031500041031092420380914F0390915003A0913C
:103160005103B091520346015701881A990AAA0ADD
:10317000BB0A82EA93E00E94780386169706A806A7
:10318000B90608F4B1C0C0924F03D0925003E09248
:103190005103F09252030E94C00180913A0388309B
:1031A000A0F08091EB039091EC03A091ED03B0911E
:1031B000EE035CE1B695A795979587955A95D1F75B
:1031C000892B8A2B8B2B09F0C4C180913A038F5F26
:1031D00080933A0380914B0390914C03A0914D034F
:1031E000B0914E030097A105B105F1F0C81AD90AB4
:1031F000EA0AFB0A82EA93E00E9478036C157D05D7
:103200008E059F0508F01BC18091EB0384FD04C06F
:1032100080ED97E00E94FF0210924B0310924C0346
:1032200010924D0310924E0390910203907C909364
:1032300002035091CE028091CF022091CD02581707
:1032400009F41AC1223009F017C190589093020373
:10325000E091CA03E770F0E0E45EFD4F6081693001
:1032600008F0F2C0615040E04613F0C08093CF02F6
:1032700087E3840F90910203892B8093020340938C
:10328000D00283E08093CD02469A1091AF038091E3
:10329000590381113EC18091EB0382FD46C1812F0C
:1032A0000E94FE0580915A030E943705E091CA03EF
:1032B000E770F0E0E45EFD4F608182E093E00E9401
:1032C00019078091EB0382FD39C1E0915A03EF5F4A
:1032D000E0935A03E83109F439C1F0E0EE55FC4FB0
:1032E0008785882309F432C10E948807813069F5F7
:1032F0008091CA03887149F180913D0390913E030A
:10330000880F991F90933E0380933D0383E0809341
:103310009F030E94DE060E94101B60933F03709380
:1033200040038093410390934203672B682B692BE2
:1033300061F481E090E0A0E0B0E080933F039093DF
:103340004003A0934103B09342038091CA0384FFDA
:103350002BC080914B0390914C03A0914D03B091F1
:103360004E03892B8A2B8B2BF9F080913D03909192
:103370003E038E7F0E94AE04182F60913B03809124
:1033800046030E94400B482F612F8091450349A3BB
:103390000E94400B00910004282F49A16091430333
:1033A000809144030E9454174698809157038130BE
:1033B000C1F018F08230B1F1D9C082E10E94541CF2
:1033C000892B09F0D3C081E0809357030E94041B2E
:1033D0006093530370935403809355039093560363
:1033E000C5C082E10E94541C892B31F50E94041B48
:1033F000C0905303D0905403E0905503F0905603CF
:103400006C197D098E099F09693E734081059105FC
:1034100008F4ACC082E08093570380ED97E00E94EF
:10342000FF02A4C082E10E94541C892B09F49EC0B3
:1034300080E090E00E94FF021092570397C080E066
:1034400090E00E94FF02F0CE68E00DCF851709F4EE
:103450000DCF4F5F242F30E090E0F901EE5FFC4F7D
:10346000DC01A752BD4F7C917083F901E053FD4F01
:10347000708301968F71F8CE2430B1F42091D00280
:1034800081ED92E0A3E0B3E0FC013E2F381B321740
:1034900018F431913D93F9CF87E3820F90910203A5
:1034A000892B80930203EDCE80915703823051F433
:1034B0009160909302035F9A8E010F5F1F4FF12C72
:1034C000B80110C05F988091CD02811103C081E0E6
:1034D0008093CD028091CD02833071F784E0809398
:1034E000CD02EACF8F2D69A37AA30E94690DF8015E
:1034F000819391938F01F39469A17AA1F0E1FF1276
:10350000F1CF8091CA0343E053E087700E94FD032E
:10351000BBCE112309F4BFCE9091580321E0290FAF
:10352000209358039813B7CE1DC082E00E94541C0C
:10353000892B09F0B4CE5F9A17E0B1CE82E00E94E9
:10354000541C892B09F0C1CE5F98BFCE10925A034C
:10355000CBCE80913A03883009F45F9A89E080935A
:103560003A03C2CE10925803115095CEA296ECE0C9
:103570000C943A261F920F920FB60F9211242F939C
:103580003F938F939F93AF93BF9380910204909149
:103590000304A0910404B09105043091010423E0D8
:1035A000230F2D3720F40196A11DB11D05C026E87B
:1035B000230F0296A11DB11D2093010480930204E4
:1035C00090930304A0930404B0930504809106042F
:1035D00090910704A0910804B09109040196A11DDF
:1035E000B11D8093060490930704A0930804B09340
:1035F0000904BF91AF919F918F913F912F910F90AF
:103600000FBE0F901F9018952FB7F8946091020489
:103610007091030480910404909105042FBF0895D4
:103620003FB7F8948091060490910704A091080494
:10363000B091090426B5A89B05C02F3F19F001964B
:10364000A11DB11D3FBF6627782F892F9A2F620FCA
:10365000711D811D911D42E0660F771F881F991F04
:103660004A95D1F70895CF92DF92EF92FF92CF93D0
:10367000DF936B017C010E94101BEB01C114D1048C
:10368000E104F10479F00E94101B6C1B7D0B683E75
:103690007340A0F381E0C81AD108E108F108C851CD
:1036A000DC4FECCFDF91CF91FF90EF90DF90CF9088
:1036B0000895789484B5826084BD84B5816084BDAA
:1036C00085B5826085BD85B5816085BDEEE6F0E09B
:1036D000808181608083E1E8F0E0108280818260F7
:1036E0008083808181608083E0E8F0E08081816078
:1036F0008083E1E9F0E08081826080838081816065
:103700008083E0E9F0E0808181608083E1ECF0E09B
:1037100080818460808380818260808380818160F9
:103720008083E3ECF0E0808181608083E0ECF0E076
:10373000808182608083E2ECF0E080818160808320
:10374000EAE7F0E08081846080838081826080830A
:10375000808181608083808180688083089590E08B
:10376000FC013197EE30F10590F5E35AFF4F0C94D0
:103770004F26809180008F7703C0809180008F7DDD
:1037800080938000089584B58F7702C084B58F7DC3
:1037900084BD0895809190008F7707C0809190003C
:1037A0008F7D03C080919000877F80939000089563
:1037B0008091C0008F7703C08091C0008F7D80937F
:1037C000C00008958091C200877F8093C200089551
:1037D000CF93DF9390E0FC01E75EFE4F2491FC0164
:1037E000E95CFE4F8491882349F190E0880F991F8E
:1037F000FC01EF58FE4FA591B4918D599E4FFC01ED
:10380000C591D4919FB7611108C0F8948C9120950F
:1038100082238C93888182230AC0623051F4F89409
:103820008C91322F309583238C938881822B8883CF
:1038300004C0F8948C91822B8C939FBFDF91CF9121
:103840000895A1E0B0E0E7E2FCE10C942626282FE1
:1038500030E0F901E550FF4F8491F901E75EFE4F3A
:103860001491F901E95CFE4F04910023C9F088230B
:1038700021F069830E94AF1B6981E02FF0E0EE0F19
:10388000FF1FED59FE4FA591B4919FB7F8948C910D
:10389000611103C01095812301C0812B8C939FBFC0
:1038A0002196E4E00C944226CF93DF93282F30E05A
:1038B000F901E550FF4F8491F901E75EFE4FD49185
:1038C000F901E95CFE4FC491CC2391F081110E9473
:1038D000AF1BEC2FF0E0EE0FFF1FEB5AFE4FA59150
:1038E000B4912C912D2381E090E021F480E002C07E
:1038F00080E090E0DF91CF910895809158049091FD
:10390000590420915A0430915B04821B930B8F73EE
:1039100099270895209158043091590480915A04B0
:1039200090915B042817390749F0E0915A04F0910F
:103930005B04E85EFB4F808190E008958FEF9FEF7E
:103940000895209158043091590480915A0490911F
:103950005B0428173907A9F0E0915A04F0915B0441
:10396000E85EFB4F808120915A0430915B042F5F09
:103970003F4F2F73332730935B0420935A0490E01A
:1039800008958FEF9FEF0895CF93DF93C091580470
:10399000D09159042196CF73DD2780915A049091DC
:1039A0005B04C817D90799F082E00E9479218F3F04
:1039B0002FEF920761F0E0915804F0915904E85E0E
:1039C000FB4F8083D0935904C0935804DFCFDF911D
:1039D000CF91089583E00E94C4230895A1E0B0E050
:1039E000E4EFFCE10C9426268C0169838091A4010C
:1039F000882359F041E050E0BE016F5F7F4F83E0C4
:103A00000E94AC21181619063CF081E090E0F80104
:103A10009383828380E090E02196E4E00C94422638
:103A2000FC0120812E5F208342E450E06FE771E0CB
:103A300080E80E942C220895FC0181819081913AB6
:103A400059F4813209F04BC047E050E06DE971E074
:103A500080E00E942C2245C0913209F040C08032A3
:103A600039F467E070E08DE991E00E94702239C07E
:103A7000823209F034C082818093A40180919D013B
:103A800090919E01A0919F01B091A001803B944034
:103A9000A105B10531F58091A40180FD12C087E731
:103AA00097E790930108809300082BE088E190E06D
:103AB0000FB6F894A895809360000FBE2093600025
:103AC00010C088E10FB6F8948093600010926000F7
:103AD0000FBEA895109201081092000802C080E065
:103AE000089581E00895089510920D0410920C0439
:103AF00088EE93E0A0E0B0E080930E0490930F0472
:103B0000A0931004B09311048EE292E090930B0402
:103B100080930A040895A0E0B0E0E1E9FDE10C948F
:103B200022266C017A01EB01E60EF71E00E010E0A0
:103B3000CE15DF0561F06991D601ED91FC91019000
:103B4000F081E02DC6010995080F191FF1CFC801BA
:103B5000CDB7DEB7E8E00C943E266115710589F01B
:103B6000DB010D900020E9F7AD0141505109461BE2
:103B7000570BDC01ED91FC910280F381E02D09955A
:103B8000089580E090E00895EF92FF920F931F93C5
:103B9000CF93DF938C01FB01C0E0D0E064917F0103
:103BA0008FEFE81AF80A662361F0D801ED91FC91D5
:103BB0000190F081E02DC8010995C80FD91FF701C8
:103BC000EDCFCE01CDB7DEB7E6E00C9440260E94E3
:103BD000AD1D0895DC01ED91FC910190F081E02D87
:103BE000099508950F931F93CF93DF93EC016DE038
:103BF0000E94EA1D8C016AE0CE010E94EA1D800F3E
:103C0000911FDF91CF911F910F9108950F931F93F3
:103C1000CF93DF93EC010E94C41D8C01CE010E9462
:103C2000F21D800F911FDF91CF911F910F91089589
:103C30000F931F93CF93DF93EC010E94AD1D8C0176
:103C4000CE010E94F21D800F911FDF91CF911F9135
:103C50000F9108950F931F93CF93DF93EC010E9470
:103C6000EA1D8C01CE010E94F21D800F911FDF9191
:103C7000CF911F910F910895A1E2B0E0E2E4FEE13F
:103C80000C941E267C01C42EE52FCB01D22E19A246
:103C900021E02D1510F02AE0D22E8E010F5D1F4F6E
:103CA0008D2C912CA12CB12C6C2D7E2FA501940173
:103CB0000E94D7258C2DD29E801911240150110904
:103CC0008A3010F4805D01C0895CF8018083211581
:103CD00031054105510521F0C22EE32FCA01E4CF81
:103CE000B801C7010E94AD1DA196ECE00C943A26E4
:103CF000A0E0B0E0EEE7FEE10C942226EC016A01C0
:103D00007B012115310541F4E881F9810190F081B1
:103D1000E02D642F09951DC02A303105A9F477FFE5
:103D200012C06DE20E94EA1D8C0144275527BA019A
:103D30004C195D096E097F092AE0CE010E943C1EE4
:103D4000800F911F06C02AE0B701A601CE010E9494
:103D50003C1ECDB7DEB7E8E00C943E260F931F93D0
:103D6000CF93DF93EC019A01AB01662757FD609575
:103D7000762F0E94781E8C01CE010E94F21D800FCA
:103D8000911FDF91CF911F910F910895211531055A
:103D900049F4DC01ED91FC910190F081E02D642F5C
:103DA000099508950E943C1E08959A01462F50E0FF
:103DB00060E070E00E94C61E08959A01AB0160E0C9
:103DC00070E00E94C61E08950F931F93CF93DF9358
:103DD000EC019A01462F50E060E070E00E94C61EA0
:103DE0008C01CE010E94F21D800F911FDF91CF91B7
:103DF0001F910F910895FC0124853585F901E05C40
:103E0000FF4F80819181F901EE5BFF4F208131816D
:103E1000821B930B8F7399270895FC0184859585E8
:103E2000FC01E05CFF4F40815181FC01EE5BFF4FE4
:103E3000208131814217530741F00190F081E02D3C
:103E4000E80FF91F808190E008958FEF9FEF0895AC
:103E5000FC0184859585FC01E05CFF4F4081518128
:103E6000FC01EE5BFF4F208131814217530779F04F
:103E7000A081B181A80FB91F8C91208131812F5F62
:103E80003F4F2F7333273183208390E008958FEFC6
:103E90009FEF0895FC0181A1882329F0A489B589A9
:103EA0008C9186FFFBCF11A20895CF93DF93FC0185
:103EB00026853785D901A05CBF4F8D919C911197C4
:103EC00001968F739927E901CE5BDF4F48815981B5
:103ED00084179507D9F30D90BC91A02DA20FB31FA5
:103EE0006C93A685B785A05CBF4F11969C938E936B
:103EF000A689B7892C9181E090E0078C02C0880FD9
:103F0000991F0A94E2F7282B2C9381E081A304885F
:103F1000F589E02D80818064808381E090E0DF91ED
:103F2000CF91089508951F920F920FB60F9211240A
:103F30002F933F934F938F939F93EF93FF93809192
:103F4000C80082FD1CC04091CE0080910205909176
:103F5000030501968F73992720910405309105057B
:103F60008217930771F0E0910205F0910305EE537B
:103F7000FB4F4083909303058093020502C080911C
:103F8000CE00FF91EF919F918F914F913F912F9193
:103F90000F900FBE0F901F9018958CE594E00E9433
:103FA000FB1E892B11F00E94921F08951F920F9201
:103FB0000FB60F9211242F933F938F939F93EF93FC
:103FC000FF932091BE043091BF048091C004909172
:103FD000C1042817390731F48091C9008F7D80937F
:103FE000C90014C0E091C004F091C104E258FB4F35
:103FF00020818091C0049091C10401968F7399270C
:104000009093C1048093C0042093CE00FF91EF9160
:104010009F918F913F912F910F900FBE0F901F9006
:104020001895A0E0B0E0E7E1F0E20C941E26FC0158
:104030001382128288EE93E0A0E0B0E0848395833F
:10404000A683B78380E492E0918380837587648739
:1040500057874687318B208B138B028BF58AE48A36
:10406000D78AC68AB18EA08E938E828E8F85848FDA
:104070008889858F8989868F8A89878F8B8980A394
:10408000ECE00C943A26CF92DF92EF92FF92CF931E
:10409000DF93EC016A017B01411581EE5807610550
:1040A0007105F9F0EC89FD8981E090E008A002C07B
:1040B000880F991F0A94E2F7808360E079E08DE32E
:1040C00090E0A70196010E94D725215031094109AE
:1040D00051095695479537952795211580E1380761
:1040E00098F0EC89FD89108260E874E88EE190E038
:1040F000A70196010E94D725215031094109510994
:104100005695479537952795E889F9893083EA8947
:10411000FB89208319A2EE89FF89408181E090E02C
:104120009C010C8C02C0220F331F0A94E2F7422B31
:104130004083EE89FF8940819C010D8C02C0220FD3
:10414000331F0A94E2F7422B4083EE89FF894081B6
:104150009C010E8C02C0220F331F0A94E2F7422BFF
:104160004083EE89FF8920810F8C02C0880F991F40
:104170000A94E2F7809582238083DF91CF91FF90AC
:10418000EF90DF90CF9008958F929F92AF92BF9261
:10419000CF92DF92EF92FF920F931F9381E08F9364
:1041A00085E08F9387E08F9383E08F9384E08F93F4
:1041B000EEEC8E2E912CFAECAF2EB12CA9ECCA2E7F
:1041C000D12CB8ECEB2EF12C0CEC10E02DEC30E007
:1041D0004EE754E062EC74E08CE594E00E9411201C
:1041E0000F900F900F900F900F901F910F91FF90D5
:1041F000EF90DF90CF90BF90AF909F908F900895F9
:104200000E94591B86E095E00E94CE230E9405156E
:10421000CDECDFE10E94A7172097E1F30E94CD1FAC
:10422000F9CF615030F02091F100FC01208301961C
:10423000F8CF289884E680930D0508952FB7FC01E8
:104240002083F89467706093E9000895A1E0B0E0DE
:10425000ECE2F1E20C942826682FCE0101960E9430
:104260001E218091F20099819FBF2196E2E00C947B
:104270004426A2E0B0E0EFE3F1E20C942526F62E0E
:104280008A0190910C05992311F057FF03C08FEF1D
:104290009FEF2BC0682FCE0101967A830E941E21CA
:1042A0008091F20090E0A8017A81801791070CF4C8
:1042B000AC01EF2DF72FF40E84E6FE1639F02898A6
:1042C00080930D059091F1009193F7CF4115510521
:1042D00021F08091F200882321F089818FBFCA01EB
:1042E00004C08BE68093E800F8CF2296E5E00C94BA
:1042F0004126A1E0B0E0EFE7F1E20C94282641E08E
:1043000050E0BE016F5F7F4F0E943921019719F481
:10431000898190E002C08FEF9FEF2196E2E00C943C
:104320004426A1E0B0E0E7E9F1E20C942826682FEA
:10433000CE0101960E941E219091E800892F807283
:1043400095FF04C09091F20080E4891B99819FBF82
:104350002196E2E00C944426A1E0B0E0E2EBF1E229
:104360000C941A26582E7B01A42E952E80910C05B4
:10437000882369F0042F152F8AEFB82E852D8072BF
:10438000782E9AE3892E852D8074682E11C08FEFC8
:104390009FEF53C0852D0E949121482E81110CC0A2
:1043A000BA94A9F361E070E080E090E00E94331BD2
:1043B0000115110579F737C0282F30E002171307D0
:1043C0000CF4402EC42CD12C0C191D09652DCE01E6
:1043D00001960E941E21772039F04A948FEF4816EB
:1043E000B1F01092F100F9CFF701842D57FE07C00C
:1043F000815058F094919093F1003196F9CF81500B
:1044000020F091919093F100FACFEC0CFD1C80917B
:10441000E80085FF0FC00115110511F461100AC0F5
:1044200089818FBFC5CF5D9884E680930E058A2D64
:10443000992D03C08092E800F3CF2196E0E10C941F
:1044400036261092E90010920B0510920A059093FF
:104450000905809308050895CF93DF93FB0120E0C1
:1044600030E0DEEF24173507A1F187FF02C0C491C9
:1044700001C0C081A0910A05B0910B0560910805AB
:1044800070910905A617B707B4F49091E8009570EC
:10449000E1F39091E80092FD1EC0C093F10060919D
:1044A0000A0570910B056F5F7F4F6F737727672B3E
:1044B00011F4D093E80060910A0570910B056F5FCD
:1044C0007F4F70930B0560930A052F5F3F4F319626
:1044D000C9CFC90102C08FEF9FEFDF91CF9108953F
:1044E000A1E0B0E0E6E7F2E20C942726162F209137
:1044F000E80022FFFCCF612F79830E9411218BEF0E
:104500008093E800812F7981972F2196E3E00C9426
:104510004326A1E0B0E0EFE8F2E20C9428261982ED
:10452000CE0101960E94101DCE0101960E946824C2
:10453000898190E02196E2E00C9444261F920F922C
:104540000FB60F921124EF92FF920F931F932F93A8
:104550003F934F935F936F937F938F939F93AF930B
:10456000BF93EF93FF93CF93DF93CDB7DEB76297FF
:10457000DEBFCDBF1092E9008091E80083FFE7C065
:1045800068E0CE010A960E94112182EF8093E80034
:104590009A8597FF05C08091E80080FFFCCF03C09B
:1045A0008EEF8093E800892F807609F0B5C08B8567
:1045B000811105C01092F1001092F100C1C0282FA6
:1045C0002D7F213009F4BCC0853049F48091E8008A
:1045D00080FFFCCF8C8580688093E300B1C086307B
:1045E00009F072C02D85E888F988223071F580E0E5
:1045F00090E02A8B0E9421220E94892299E08E015C
:104600000F5F1F4FF801392F11923A95E9F79983FF
:104610002A892A8391E09E8390E898879AEF998768
:1046200020910A0530910B05275F3F4F3C832B8378
:104630008D83C7010E94212249E050E0B80180E04B
:104640000E942C220E9489227BC0C7012A8B0E94D3
:1046500021222A89223241F482E290E00E947424CD
:10466000892B09F06DC070C0213069F4888999895F
:10467000089711F42093070580910705882389F096
:1046800066EC71E016C0233009F05EC08C8588238B
:1046900059F0823061F0813009F056C06AEE71E065
:1046A00008C068ED71E005C064E272E002C062E03B
:1046B00072E06115710509F447C0FB01449150E0B7
:1046C00080E80E942C223CC0873009F43DC088302D
:1046D00021F481E08093F10033C0893089F5937033
:1046E00099F5E2ECF1E081E021E096E38093E900C6
:1046F0002093EB0034913093EC009093ED008F5FAA
:104700003196853099F78EE78093EA001092EA009F
:104710008C8580930C0514C0888999890E94212278
:104720008E85811105C0CE010A960E941C1D06C00F
:10473000823051F4CE010A960E949624882321F0FB
:104740008EEF8093E80003C081E28093EB006296D5
:104750000FB6F894DEBF0FBECDBFDF91CF91FF91B2
:10476000EF91BF91AF919F918F917F916F915F91E9
:104770004F913F912F911F910F91FF90EF900F90CC
:104780000FBE0F901F9018958093E9008091F20062
:10479000882319F08AE38093E800089510920C05AD
:1047A00081E08093D70080EA8093D80082E189BDC0
:1047B00009B400FEFDCF61E070E080E090E00E946F
:1047C000331B80E98093D8008CE08093E200109244
:1047D000E000559A209A08951F920F920FB60F92FB
:1047E00011242F933F934F935F936F937F938F93F6
:1047F0009F93AF93BF93EF93FF938091E10010924B
:10480000E10083FF0FC01092E90091E09093EB006C
:104810001092EC0092E39093ED0010920C0598E05A
:104820009093F00082FF26C083E00E94C42382E0C0
:104830000E942621882321F08AE094E00E94C41C73
:1048400080910E05882339F080910E058150809368
:104850000E05882369F080910D05882359F0809119
:104860000D05815080930D05811104C0289A02C066
:104870005D9AF1CFFF91EF91BF91AF919F918F9191
:104880007F916F915F914F913F912F910F900FBE4C
:104890000F901F901895FF920F931F93CF93DF9364
:1048A000EC01F62EE881F9810480F581E02D09956F
:1048B0008C01E881F9810680F781E02D6F2DCE0112
:1048C0000995C8019927CDB7DEB7E5E00C944126DC
:1048D000FC0120812F5F208349E150E068EA72E00B
:1048E00080E80E942C22089545E650E061EC72E0D9
:1048F00080E80E942C220895A1E0B0E0E2E8F4E212
:104900000C94242689838B017A0141E050E0BE019A
:104910006F5F7F4F84E00E94AC21A701B80184E45F
:104920000E94AC212196E6E00C944026FC01918186
:104930008081813A31F481E0913091F0933089F4B3
:1049400011C0813271F49B3021F482818093A601E1
:1049500005C09A3031F482818093A50181E00895E9
:10496000089580E00895FC0110820895FC011382EF
:10497000128220E532E031832083089548E050E040
:1049800082E00E947C240895CF93DF93DC01683895
:1049900018F0E8E7E60F25C0E62FF0E067FF11C04A
:1049A000E058F10981E090E001C0880FEA95EAF74C
:1049B00014969C911497982B14969C931497E0E06E
:1049C00010C0E85DFD4FE491EE2309F440C0E7FF1D
:1049D00008C014968C911497826014968C93149747
:1049E000EF7716968C9116978E1741F117968C914A
:1049F00017978E1719F118968C9118978E17F1F05A
:104A000019968C9119978E17C9F01A968C911A974E
:104A10008E17A1F01B968C911B978E1779F080E072
:104A200090E0ED01C80FD91F2E81211102C0EE8345
:104A300005C0019686309105A1F709C0BD016C5FE4
:104A40007F4FCD010E94BE2481E090E008C081E04C
:104A500090E013969C938E93129780E090E0DF9104
:104A6000CF910895683818F0E8E7E60F25C0E62FE3
:104A7000F0E067FF12C0E058F10921E030E001C02A
:104A8000220FEA95EAF72095DC0114963C911497E1
:104A9000322314963C93E0E00FC0E85DFD4FE491B3
:104AA000EE2329F1E7FF08C0DC0114962C9114973E
:104AB0002D7F14962C93EF7720E030E0EE2351F019
:104AC000DC01A20FB31F16964C9116974E1302C02D
:104AD00016961C922F5F3F4F2630310579F7BC01A7
:104AE0006C5F7F4F0E94BE2481E090E0089580E0DB
:104AF00090E00895FC0116821782108611861286B6
:104B000013861482BC016C5F7F4F0E94BE240895FF
:104B10008BE195E00E94B3248FE095E00E94B624DB
:104B20000895A29FB001B39FC001A39F700D811D86
:104B30001124911DB29F700D811D1124911D0895A6
:104B40000E949125A59F900DB49F900DA49F800D6C
:104B5000911D11240895B7FF0C94A0250E94A02553
:104B6000821B930B0895DB018F939F930E94A025D6
:104B7000BF91AF91A29F800D911DA39F900DB29FF9
:104B8000900D1124089597FB072E16F4009407D07A
:104B900077FD09D00E94552607FC05D03EF490957C
:104BA00081959F4F0895709561957F4F0895A1E27B
:104BB0001A2EAA1BBB1BFD010DC0AA1FBB1FEE1F97
:104BC000FF1FA217B307E407F50720F0A21BB30BE2
:104BD000E40BF50B661F771F881F991F1A9469F75E
:104BE00060957095809590959B01AC01BD01CF01BA
:104BF0000895052E97FB1EF400940E94102657FD81
:104C000007D00E94D72507FC03D04EF40C94102641
:104C100050954095309521953F4F4F4F5F4F0895E8
:104C200090958095709561957F4F8F4F9F4F089518
:104C30002F923F924F925F926F927F928F929F92AC
:104C4000AF92BF92CF92DF92EF92FF920F931F939A
:104C5000CF93DF93CDB7DEB7CA1BDB0B0FB6F8944B
:104C6000DEBF0FBECDBF09942A88398848885F848B
:104C70006E847D848C849B84AA84B984C884DF80FC
:104C8000EE80FD800C811B81AA81B981CE0FD11DE0
:104C90000FB6F894DEBF0FBECDBFED010895EE0F45
:104CA000FF1F0590F491E02D0994AA1BBB1B51E155
:104CB00007C0AA1FBB1FA617B70710F0A61BB70B8C
:104CC000881F991F5A95A9F780959095BC01CD0131
:104CD00008958F929F92AF92BF92CF92DF92EF9200
:104CE000FF92CF93DF93EC01688179818A819B8168
:104CF000611571058105910521F464E279ED8BE57B
:104D000097E02DE133EF41E050E00E94F9254901A1
:104D10005A019B01AC01A7EAB1E40E94A0256B01F6
:104D20007C01ACEEB4EFA50194010E94AE25C60E45
:104D3000D71EE81EF91EF7FE06C081E0C81AD1088A
:104D4000E10880E8F80AC882D982EA82FB82C701BA
:104D5000B6019F77DF91CF91FF90EF90DF90CF90DA
:104D6000BF90AF909F908F9008950E9469260895FC
:104D700086E091E00E946926089560930601709391
:104D8000070180930801909309010895F999FECFD6
:104D900092BD81BDF89A992780B50895262FF9997B
:104DA000FECF1FBA92BD81BD20BD0FB6F894FA9A0E
:0C4DB000F99A0FBE01960895F894FFCF09
:104DBC0000001C05200001000000FF0002000200A2
:104DCC0002000200020002000200020002000200C7
:104DDC000200020002000200020002802500000511
:104DEC00400AA1204EA50020244EA52C2330C01231
:104DFC0000001A400AA1204EA5001B1E27522C238E
:104E0C00308025000005400AA1204EA50020244E2C
:104E1C00A52C2330004B000006400AD0009D490011
:104E2C007B289D492C233000E1000005400A4501F8
:104E3C00D7DC03B81E0EBF00232E48E801008A40C1
:104E4C000A6001555502AD1E20000023C800E10088
:104E5C000000000000010154582074696D656F75E5
:104E6C00742100456E746572696E672061646170AF
:104E7C0074697665206368616E6E656C2073656C11
:104E8C00656374696F6E2C207069636B696E673A29
:104E9C00007363616E6E6572206D6F6465004F7098
:104EAC00656E4C52536E6720545820737461727443
:104EBC00696E672000206F6E20485720006D6F646C
:104ECC00756C65206C6F636B65643F0000070B0CA1
:104EDC0010111500160A1322312900000000EE1CD7
:104EEC008B1D7D1CA11C8A1CEA1CC41C000000002C
:104EFC00551F8B1DFB1E281F0D1F4A1F0000000095
:0A4F0C004B248B1DC42432257A25A6
:1070000055C000006EC000006CC000006AC00000E7
:1070100068C0000066C0000064C0000062C00000DC
:1070200060C000005EC00000F2C400005AC0000052
:1070300058C0000056C0000054C0000052C00000FC
:1070400050C0000078C000004CC000004AC00000E2
:1070500048C0000046C0000044C0000042C000001C
:1070600040C000003EC000003CC000003AC000002C
:1070700038C0000036C0000034C0000032C000003C
:1070800030C000002EC000002CC000002AC000004C
:1070900028C0000026C0000024C0000022C000005C
:1070A00020C000001EC000001CC0000011241FBE34
:1070B000CFEFDAE0DEBFCDBF11E0A0E0B1E0E2E368
:1070C000FFE702C005900D92A83AB107D9F711E089
:1070D000A8EAB1E001C01D92AE3BB107E1F78FD342
:1070E00026C78ECFF89410926F00109281001092F4
:1070F00085001092840081E085BF15BE47985D9A97
:10710000289A0C94000008952091B2013091B301A7
:107110002F5F3F4F3093B3012093B201932F37FF7E
:1071200003C08EEF831B982F990F921710F4479886
:107130000895479A08951F920F920FB60F92112447
:107140002F938F939F93EF93FF931092850010924C
:1071500084008091A8019091A901009741F00197C6
:107160009093A9018093A801892B09F45D9A8091DD
:10717000AA019091AB01009741F001979093AB0168
:107180008093AA01892B09F4289AE0E0F0E0859128
:1071900094918F5F9F4F49F08091AC019091AD0128
:1071A00001969093AD018093AC01FF91EF919F9177
:1071B0008F912F910F900FBE0F901F90189584E024
:1071C0008093E9000DC08091E8008B778093E80000
:1071D00003C08EB3882351F08091E80082FFF9CF7D
:1071E0008091E80085FFEFCF8091F1000895982FFE
:1071F00083E08093E9008091E80085FD0DC08091D7
:10720000E8008E778093E80003C08EB3882369F08E
:107210008091E80080FFF9CF9093F1005D9884E6BB
:1072200090E09093A9018093A80108954F925F92F6
:107230006F927F928F929F92AF92BF92CF92DF9286
:10724000EF92FF920F931F93CF93DF9384E080938D
:10725000E9008091E80082FF57C2289884E690E018
:107260009093AB018093AA01AADF182F853481F493
:107270008CE49DE19093AD018093AC0107B600FCD6
:10728000FDCFF999FECF81E180935700E89503C0C7
:10729000843519F494DF8DE00DC28C34E1F3803530
:1072A000D1F3843721F484E4A2DF80E003C2813685
:1072B00011F489E5FFC18134B1F481DF182F7FDF3C
:1072C00090E0880F991FAA2797FDA095BA2F312F1C
:1072D000330F20E0442737FD4095542F822B932B0A
:1072E000A42BB52BB8C1803711F483E5E3C18335F6
:1072F00049F4C0E0D1E089917ADF21E0C730D207BC
:10730000D1F7D9C1863521F481E371DF80E3D2C1A1
:10731000833731F487E86BDF85E969DF8EE1CAC125
:107320008536B9F4E0E0F0E093E085E09093570013
:10733000E89507B600FCFDCF80935700E89507B6A7
:1073400000FCFDCFE058FF4FA0E7E030FA0771F7EF
:10735000A2CF823739F4E1E0F0E089E08093570072
:107360008491A8C1863439F4E0E0F0E089E08093AC
:10737000570084919FC18E3439F4E3E0F0E089E056
:1073800080935700849196C1813539F4E2E0F0E0B2
:1073900089E08093570084918DC1823631F489E56C
:1073A00026DF80E024DF80E885C1823419F087364B
:1073B00009F0E5C01092AD011092AC0100DF082F7A
:1073C000FEDEF82EFCDE682E8554823008F071C196
:1073D000902F80E0CF2DD0E0C82BD92B10926F00DA
:1073E000173609F04BC081E180935700E895DD2402
:1073F000CC24C3943FC0E090AE01F090AF01009167
:10740000B0011091B101B6E46B16D9F4ED2DF0E0A6
:10741000EE29FF29E4918E2FEADEDD2081F082E063
:1074200090E0A0E0B0E0E80EF91E0A1F1B1FE092FA
:10743000AE01F092AF010093B0011093B101DC24D2
:1074400018C0D801C701B695A7959795879559D5C6
:10745000CEDE82E090E0A0E0B0E0E80EF91E0A1F68
:107460001B1FE092AE01F092AF010093B0011093A8
:10747000B1012197209709F0BECF7DC08090AE0169
:107480009090AF01A090B001B090B10196E4691660
:1074900009F05DC083E0F40180935700E89507B6DA
:1074A00000FCFDCF54C0F6E46F1661F5772031F192
:1074B000E090AE01F090AF010091B0011091B101E8
:1074C0007EDED82ECC24852D90E08C299D29F701D5
:1074D0000C0140925700E895112482E090E0A0E072
:1074E000B0E0E80EF91E0A1F1B1FE092AE01F092F9
:1074F000AF010093B0011093B10102C060DE582EBD
:10750000742423C0E090AE01F090AF010091B0016F
:107510001091B10116950795F794E79450DE682F06
:10752000C701F7D48091AE019091AF01A091B00155
:10753000B091B1010296A11DB11D8093AE0190934F
:10754000AF01A093B001B093B101219704C05524BD
:10755000772444244394209709F0A5CF96E4691634
:1075600041F485E0F40180935700E89507B600FCEC
:10757000FDCF8DE03CDE82E080936F009CC08334C1
:1075800071F40091AE011091AF0119DE90E021E09D
:10759000F8010C0120935700E89511247CCE833626
:1075A00019F5E090AE01F090AF010091B00110919B
:1075B000B10105DEF701E16090E021E00C012093CC
:1075C0005700E895112482E090E0A0E0B0E0E80EDA
:1075D000F91E0A1F1B1FE092AE01F092AF0100934B
:1075E000B0011093B10157CE8D3661F4E091AE0138
:1075F000F091AF0185E080935700E89507B600FC55
:10760000FDCF49CE823551F4E091AE01F091AF014A
:1076100005911491812FEBDD802F4CC0843421F52E
:10762000E090AE01F090AF010091B0011091B10176
:1076300016950795F794E794C2DD682FC70169D4C2
:107640008091AE019091AF01A091B001B091B101D4
:107650000296A11DB11D8093AE019093AF01A0933E
:10766000B001B093B10117CE843609F5E090AE01B8
:10767000F090AF010091B0011091B101D801C701A4
:10768000B695A795979587953CD4B1DD82E090E0BB
:10769000A0E0B0E0E80EF91E0A1F1B1FE092AE0149
:1076A000F092AF010093B0011093B10104C08B318F
:1076B00011F08FE39CDD83E08093E9009091E80076
:1076C0008091E8008E778093E80095FF04C010C099
:1076D0008EB38823C9F08091E80080FFF9CF8091B4
:1076E000E8008E778093E80003C08EB3882361F0B2
:1076F0008091E80080FFF9CF84E08093E9008091D9
:10770000E8008B778093E800DF91CF911F910F9174
:10771000FF90EF90DF90CF90BF90AF909F908F90B1
:107720007F906F905F904F9008959091B601892F50
:107730008F77813249F58091B7018032A1F0813293
:1077400019F5913A09F58091E800877F8093E80068
:107750008DE091E067E070E00BD28091E8008B77DC
:107760008093E8000895913279F48091E800877F52
:107770008093E8008DE091E067E070E05DD2809159
:10778000E8008E778093E800089582E061EC42E0A3
:10779000B5D083E061E842E1B1D084E060E842E145
:1077A000ADC084B7877F84BF88E10FB6F89480931B
:1077B0006000109260000FBE20E880E090E00FB6FD
:1077C000F89420936100809361000FBE81E085BF33
:1077D00092E095BF3F9A209A559AE1E6F0E0208327
:1077E000108247985D9A289A109289008AEF8093B8
:1077F000880090936F0083E080938100F0C04091F7
:10780000000850910108109201081092000894B7E6
:1078100014BE88E10FB6F894809360001092600067
:107820000FBE292F30E0F901E270F07091FD18C011
:1078300090FF05C0859194918F5F9F4F81F423FF46
:107840000FC08091090190910A014817590741F032
:10785000E0E0F0E0859194918F5F9F4F09F042DC6A
:10786000A0DF78941092AD011092AC010CC0DEDC68
:1078700036D38091AC019091AD0181549F4110F0BD
:107880001092140141DC80911401882381F78091CA
:10789000E00081608093E00025DC80E090E00895C6
:1078A000FA01923049F0933061F09130F9F485E1BA
:1078B00091E022E130E01EC087E291E02EE330E06B
:1078C00019C0882329F485E691E024E030E012C055
:1078D000813029F489E691E022E230E00BC0823069
:1078E00029F48DE891E028E130E004C080E090E0E8
:1078F00020E030E091838083C90108958093E900FE
:107900008091EB0081608093EB001092ED0060931A
:10791000EC004093ED008091EE00881F8827881FBF
:1079200008958091B60188238CF403C08EB3882318
:10793000B1F08091E80082FFF9CF8091E8008B7769
:107940008093E80008958EB3882349F08091E80081
:1079500080FFF9CF8091E8008E778093E80008954A
:10796000EF92FF920F931F9345D04CD008ED10E09B
:10797000F80180818F778083808180688083808117
:107980008F7D808319BC1EBA1092B40180EEE82E60
:10799000F12CF70180818B7F8083F80180818160E9
:1079A000808380E060E042E0A9DFE1EEF0E08081EA
:1079B0008E7F8083E2EEF0E0808181608083808131
:1079C00088608083F70180818E7F8083F8018081C9
:1079D000806180831F910F91FF90EF900895E7EDF4
:1079E000F0E08081816080838AE482BF81E08093BF
:1079F000B501B6CFE8EDF0E080818E7F80831092F4
:107A0000E20008951092DA001092E10008951F92AA
:107A10000F920FB60F9211242F933F934F935F93C2
:107A20006F937F938F939F93AF93BF93EF93FF9346
:107A30008091DA0080FF1BC08091D80080FF17C0C2
:107A40008091DA008E7F8093DA008091D90080FFE8
:107A50000BC080E189BD82E189BD09B400FEFDCF84
:107A600081E08EBB3BD203C019BC1EBA37D28091D5
:107A7000E10080FF17C08091E20080FF13C0809179
:107A8000E2008E7F8093E2008091E200806180932B
:107A9000E2008091D80080628093D80019BC85E014
:107AA0008EBB1CD28091E10084FF2CC08091E2004B
:107AB00084FF28C080E189BD82E189BD09B400FE50
:107AC000FDCF8091D8008F7D8093D8008091E10018
:107AD0008F7E8093E1008091E2008F7E8093E200B0
:107AE0008091E20081608093E2008091B40188235C
:107AF00031F48091E30087FD02C081E001C084E0A1
:107B00008EBBECD18091E10083FF21C08091E20027
:107B100083FF1DC08091E100877F8093E10082E0B8
:107B20008EBB1092B4018091E1008E7F8093E100C2
:107B30008091E2008E7F8093E2008091E20080617C
:107B40008093E20080E060E042E0D8DEC7D1FF91A0
:107B5000EF91BF91AF919F918F917F916F915F91C5
:107B60004F913F912F910F900FBE0F901F9018953E
:107B70009C014091BC015091BD014617570718F474
:107B8000F90190E044C06115710511F0AB01F8CF27
:107B90008091E8008E778093E80040E050E0F0CFDD
:107BA0008EB3882309F444C0853009F443C0809122
:107BB000E80083FF02C081E008958091E80082FD23
:107BC00031C08091E80080FF22C08091F300909145
:107BD000F200782F60E0292F30E0262B372B07C0EA
:107BE00081918093F100415050402F5F3F4F4115EC
:107BF000510519F02830310598F390E0283031050F
:107C000009F491E08091E8008E778093E8004115B7
:107C1000510531F6992321F605C08EB3882341F032
:107C2000853041F08091E80082FFF7CF80E0089531
:107C300082E0089583E008959C016115710529F49F
:107C40008091E8008B778093E800F90126C08EB31D
:107C5000882391F1853091F18091E80083FF02C083
:107C600081E008958091E80082FFF1CF06C0809105
:107C7000F10081936150704059F02091F3008091A0
:107C8000F200322F20E090E0822B932B892B79F7A2
:107C90008091E8008B778093E80061157105B9F653
:107CA00005C08EB3882341F0853041F08091E80013
:107CB00080FFF7CF80E0089582E0089583E0089583
:107CC0000F931F93DF93CF9300D0CDB7DEB7E6EBD2
:107CD000F1E08091F100819381E0EE3BF807C9F774
:107CE00024DD8091E80083FFE4C08091B60190918B
:107CF000B701953009F46DC0963040F4913081F1B0
:107D0000913070F0933009F0D4C02AC0983009F453
:107D1000A3C0993009F4B2C0963009F0CAC07CC043
:107D2000803809F4C6C0823809F0C3C08091BA0116
:107D300087708093E9008091EB001092E900209118
:107D4000E800277F2093E80090E025E0969587954E
:107D50002A95E1F781708093F1001092F10087C0BD
:107D6000882319F0823009F0A4C08F71823009F0A5
:107D7000A0C08091B801882331F52091BA01277005
:107D800009F497C02093E9008091EB0080FF1BC0AD
:107D9000933021F48091EB00806213C08091EB005E
:107DA00080618093EB0081E090E002C0880F991F12
:107DB0002A95E2F78093EA001092EA008091EB00A6
:107DC00088608093EB001092E9008091E800877F43
:107DD00051C0882309F06DC01091B8011F770FB70B
:107DE000F8948091E800877F8093E8009ADD809185
:107DF000E80080FFFCCF8091E3008078812B8093A6
:107E0000E30080688093E300112311F482E001C055
:107E100083E08EBB0FBF4DC08058823008F049C050
:107E20008091B8019091B9016091BA01AE014F5FA4
:107E30005F4F36DDBC01009709F43BC08091E8003C
:107E4000877F8093E80089819A8192DE8091E800A3
:107E50008B778093E8002DC0803859F58091E80039
:107E6000877F8093E8008091B4018093F100809136
:107E7000E8008E778093E80054DD1BC08823C9F4A6
:107E80009091B8019230A8F48091E800877F8093A8
:107E9000E8009093B40145DD8091B401882331F46A
:107EA0008091E30087FD02C081E001C084E08EBBC9
:107EB0006CDC8091E80083FF0AC08091EB00806257
:107EC0008093EB008091E800877F8093E8000F901B
:107ED0000F90CF91DF911F910F91089508951F93F7
:107EE0008EB3882361F01091E9001092E90080912F
:107EF000E80083FF01C0E4DE17701093E9001F91D2
:107F00000895F999FECF92BD81BDF89A992780B561
:107F10000895262FF999FECF1FBA92BD81BD20BDCD
:107F20000FB6F894FA9AF99A0FBE01960895F8944C
:107F3000FFCF4341544552494E4100777700080036
:107F400000000000000801120110010200000841B9
:107F500023360001000201000109023E0002010077
:107F60008032090400000102020100052400100112
:107F7000042402040524060001070582030800FF0B
:107F800009040100020A00000007050402100001B4
:107F90000705830210000104030904220341007253
:107FA000006400750069006E006F0020004C0065E1
:107FB000006F006E006100720064006F0000001826
:107FC00003410072006400750069006E006F0020BC
:0A7FD000004C004C004300000000CC
:00000001FF
